:1000000000308A006E2B00000A108A100A11820745
:1000100028340C34013406340A108A100A1182077D
:100020002034203445343D34253432342E343234B7
:10003000663420346C347834203420342034203436
:10004000203420342034203420340A3400340A1080
:100050008A100A1182072A342A34203420342034AA
:1000600020342034203420342034203420342034F0
:100070002034203420340D3400340A108A100A1140
:1000800082072A342A342A342A3420342034203473
:1000900020342034203420342034203420342034C0
:1000A00020340D3400340A108A100A1182072A34D1
:1000B0002A342A342A342A342A342034203420346E
:1000C00020342034203420342034203420340D34A3
:1000D00000340A108A100A1182072A342A342A347A
:1000E0002A342A342A342A342A342034203420343E
:1000F000203420342034203420340D3400340A10CD
:100100008A100A1182072A342A342A342A342A34DB
:100110002A342A342A342A342A342034203420340D
:100120002034203420340D3400340A108A100A118F
:1001300082072A342A342A342A342A342A342A34A4
:100140002A342A342A342A342A34203420342034DD
:1001500020340D3400340A108A100A1182072A3420
:100160002A342A342A342A342A342A342A342A349F
:100170002A342A342A342A342A34203420340D34C0
:1001800000340A108A100A1182072A342A342A34C9
:100190002A342A342A342A342A342A342A342A346F
:1001A0002A342A342A342A342A340D3400340A10EA
:1001B0008A100A11820720342A342A342A3420343F
:1001C00020346834693467346834203420342A3465
:1001D0002A342A3420340D3400343630840083131A
:1001E0000008031904290130F800BF30F70064004B
:1001F000F70BF728F80BF5284A30F700F70BFE2825
:1002000000006400800BF328003407080F39BD009C
:100210003C0EF700F030F7057708F0393D04870011
:100220000614831606106400831206108316061047
:1002300083120034BA08031D1F2986102029861452
:10024000831686108312BB0E3B08BC000521BB0E33
:100250003B08BC00052164000C30F700F70B2E2989
:10026000312900341430B600ED200F308316870595
:1002700083128610831686108312061083160610CA
:100280008312A7012708023C031C4E290230B60046
:10029000ED200330BC000521A70A422964000C3080
:1002A000F700F70B512954290230BC0005216400E6
:1002B0000C30F700F70B5A295D29A7012708023CEB
:1002C000031C6E2927080420A800BA012808BB00D7
:1002D0001A210230B600ED20A70A5E29C82B8E3005
:1002E000F7002808F8002708F900FA01F808031DAC
:1002F00083297908F800F9010830F702F808031D8E
:100300008329F7018B290310F81B8A29F90DF80DB1
:10031000F7038329F813DC2B35080319FC29BD00EA
:1003200039080319FC29BD0703189D297F30BD0238
:10033000031CFC290319FC29A1298130BD070318DE
:10034000FC293D08F700F801F901FA013608C1005F
:10035000C1173708C0003808BF001830BD00BE0103
:100360003F1CCA293C08FA07031CBC29F90A031DD3
:10037000BC29F80A0319BE173B08F907031CC32957
:10038000F80A0319BE173A08B700B7173708F80775
:100390000318BE17BE0DF80CF90CFA0CC10CC00CFA
:1003A000BF0C0310BD0BAF290130F7070318FC2960
:1003B000F81BE129C10DFA0DF90DF80DF70303192A
:1003C000FC29C11FF229FA0A031DF229F90A031DAB
:1003D000F229F80A031DF229F80CF90CFA0CF70AB5
:1003E0000319FC293608BE003A08BE06BE1FFA29CA
:1003F000F817002AF813002AF701F801F901FA01A9
:10040000003401303602B8003708023C031D0A2AC6
:100410004030B80738088038B900BA013908BB0045
:100420001A21003435080C3A0319202A063A031918
:10043000282A073A03192E2A053A0319332A382A9B
:10044000BA010130BB001A210230B600ED20442A67
:100450000130B6000230B7000122442A0130B60054
:10046000B7000122442ABA011030BB001A21442AE5
:1004700035081F3C031C3E2A0730B5050130BA0081
:100480003508BB001A21442A0034F701F801F901AC
:10049000FA01BD01BE01BF01C0013C083B043A04A2
:1004A00039040319832A2030C1000310B50DB60D9D
:1004B000B70DB80DBD0DBE0DBF0DC00D3C084002FF
:1004C000031D6C2A3B083F02031D6C2A3A083E02BA
:1004D000031D6C2A39083D02031C7D2A3908BD0220
:1004E0003A08031C3A0FBE023B08031C3B0FBF0235
:1004F0003C08031C3C0FC0020314F70DF80DF90D66
:10050000FA0DC10B552A3D308400831300340408D2
:10051000AD002C08AF000319A62A2B08B8002A0842
:10052000B7002908B6002808B500BC01BB0120307F
:10053000BA008230B9008C217A08AB007908AA0091
:100540007808A9007708A800AF0B8D2A2B08B800FF
:100550002A08B7002908B6002808B5003508B63CB7
:10056000B500FA013608B900B6170310B60CB70C7F
:10057000B80CFA0CF90CF80CF70CB50BB52AB91F2E
:10058000CC2AF709F809F909FA09F70A0319F80A50
:100590000319F90A0319FA0A7A08AB007908AA00C4
:1005A0007808A9007708A800AB1FE32AAD03AD16B1
:1005B000A809A909AA09AB09A80A0319A90A0319D4
:1005C000AA0A0319AB0A3B30B4009A30B300CA3010
:1005D000B200B1010A30AF002C080319AD0A2B0894
:1005E000B8002A08B7002908B6002808B500340862
:1005F000BC003308BB003208BA003108B9004522FC
:100600000008A800840A0008A900840A0008AA00BB
:10061000840A0008AB00FD308407F708031D232B74
:100620002C0A2F020319232B2D080319252B0F3910
:100630002F0203191D2B0318552BAD1B552B2D1BFA
:10064000252B2030512B2030AD05AD1E332BAD12A4
:100650002C08031DAD037708AD002D30B500122224
:100660002D08F700AD012C082F02031D412B770840
:10067000AD002E30B50012222D08F7002030AD0558
:1006800000303030AD1E512BAD122C08031DAD03D0
:100690007708AD002D30B50012222D08F700AD010E
:1006A0003030F7077708B50012223408B800330855
:1006B000B7003208B6003108B500BC01BB01BA0171
:1006C0000A30B90045227A08B4007908B3007808E6
:1006D000B2007708B100AF0BEF2A0D2C8401831311
:1006E0001F30830583161F149F141F159F11073099
:1006F0009C00FF308312A00083161F109F141F154B
:100700009F151F1383121F139F1783169F178312A2
:100710001F148316091283129412A0122008831644
:100720008700831220162008831687008312A011E9
:10073000200883168700013083129400003083164E
:1007400094000108C73908388100831290010030F5
:10075000F800920000308316920007309C000508D4
:1007600064000230F700F70BB32BB62B1C08831282
:100770000D1383169D010030F80083121F08C7393E
:1007800078049F0064000630F700F70BC52B322970
:100790001F151F19C92B83161E088312A1001E08DE
:1007A000A2006400C730F700F70BD42B000022082A
:1007B000A8002108A7006F29D630B8005630B7002E
:1007C0006C30B6007A30B5007A08BC007908BB00FE
:1007D0007808BA007708B9008C217A08A600790851
:1007E000A5007808A4007708A300A70127080C201B
:1007F000A70AF700B500122204302702031DF62BCA
:10080000893084002608AB002508AA002408A90026
:100810002308A8000230AC00872A0930A800280865
:100820000C20A80AF700B500122216302802031D7A
:100830000F2CA208031D2B2C2108803C031C2B2C01
:10084000A70127082720A70AF700B50012221130B8
:100850002702031D212CA208031D322C2108803CF5
:100860000318472C2208013C031C472C031D3C2C79
:100870002108003C031C472CA70127083D20A70A9C
:10088000F700B500122211302702031D3D2C22086B
:10089000003C0318672CFF3A031D522C2108003C32
:1008A0000318672C2208013C031C672C031D5C2CD9
:1008B0002108803C031C672CA70127085320A70AA6
:1008C000F700B500122211302702031D5D2C22080B
:1008D000003C0318872CFF3A031D722C2108803C32
:1008E0000318872C2208023C031C872C031D7C2C38
:1008F0002108003C031C872CA70127086920A70AB0
:10090000F700B500122211302702031D7D2C2208AA
:10091000013C0318A72CFF3A031D922C2108003C30
:100920000318A72C2208023C031CA72C031D9C2C97
:100930002108803C031CA72CA70127087F20A70AB9
:10094000F700B500122211302702031D9D2C22084A
:10095000013C0318C72CFF3A031DB22C2108803C30
:100960000318C72C2208033C031CC72C031DBC2CF6
:100970002108003C031CC72CA70127089520A70AC3
:10098000F700B500122211302702031DBD2C2208EA
:10099000023C0318E72CFF3A031DD22C2108003C2F
:1009A0000318E72C2208033C031CE72C031DDC2C56
:1009B0002108803C031CE72CA7012708AB20A70ACD
:1009C000F700B500122211302702031DDD2C22088A
:1009D000023C0318072DFF3A031DF22C2108803C2E
:1009E0000318072D2208033C031C072D031DFC2CB4
:1009F0002108F83C031C072DA7012708C120A70ADE
:100A0000F700B500122211302702031DFD2C220829
:100A1000023C03181D2DFF3A031D122D2108F83C3E
:100A200003181D2DA7012708D720A70AF700B50036
:100A3000122211302702031D132D0330A700C830E6
:0C0A4000B600ED20A70B1F2DC82B630093
:02400E00393F38
:00000001FF
